:100000000C9477000C94FE130C9425140C949F0010
:100010000C949F000C949F000C949F000C949F00E4
:100020000C949F000C949F000C949F000C949F00D4
:100030000C949F000C947F080C949F000C949F00DC
:100040000C944C140C949F000C9410170C944217B1
:100050000C949F000C949F000C949F000C949F00A4
:100060000C949F000C949F003B4D433D003B4D552D
:100070003D004D533D00556E737570706F72746521
:100080006420636F6D6D616E640020557365206F31
:100090006E65206F6620000000000800020100006D
:1000A0000304070000000000000000010204081023
:1000B00020408001020408102001020408102004DE
:1000C00004040404040404020202020202030303FF
:1000D00003030300000000250028002B000000009F
:1000E00000240027002A0000190872175C08112458
:1000F0001FBECFEFD8E0DEBFCDBF12E0A0E0B1E081
:10010000EAEBF7E402C005900D92A631B107D9F7EA
:1001100024E0A6E1B2E001C01D92A33EB207E1F7E0
:1001200010E0CCEED0E004C02297FE010E94FC1D3E
:10013000C83ED107C9F70E94B9170C94D0230C947C
:100140000000CF92DF92EF92FF920F931F930E94D5
:10015000A21400911D0210911E0220911F023091E5
:1001600020026B017C01C01AD10AE20AF30A97014E
:10017000860160931D0270931E0280931F0290936C
:1001800020020A3511052105310578F181E0C816F4
:100190008DE7D806E104F10410F4960102C021E0D5
:1001A0003DE74A9B03C03195219531098091630356
:1001B0008B34D8F4809163038F5F809363038091C5
:1001C0006403609162030E94A41D90936403E09114
:1001D0006403F0E0EE0FFF1FEA59FC4F31832083E8
:1001E000809164038F5F809364031F910F91FF9050
:1001F000EF90DF90CF9008950F931F9360912702A7
:100200008DE00E949515109227020E94A214009181
:100210001D0210911E0220911F0230912002601BCE
:10022000710B820B930B62307D478105910520F0A5
:100230001F910F910C94A1001F910F91089581E2DD
:1002400092E00E9461198BE593E00E94611985E5B7
:1002500093E00C946119CF93DF93EC01FB012481AF
:1002600035810E94A41BCE01DF91CF91089541E01A
:1002700050E061EA70E080E00C94CC1380E00C94D4
:10028000EC13CF93DF931F92CDB7DEB72B9A20915B
:10029000060130910701482F429FC001439F900DF6
:1002A000112469830E94ED142B988091060190918E
:1002B00007016981FC016E9FC0016F9F900D1124A1
:1002C0000F90DF91CF910C94ED14EF92FF920F936A
:1002D0001F93CF93DF93F82EE92E0E943E0100E09A
:1002E00010E02091080130E0021713072CF56FE1B0
:1002F00081E00E944101CF2DDE2D29912223C9F0FA
:10030000213371F0263449F02033B9F763E081E0FE
:100310000E94410163E081E009C063E081E002C026
:1003200061E083E00E94410161E083E00E944101BD
:10033000E4CF0F5F1F4FD5CFDF91CF911F910F916A
:10034000FF90EF900C9437013F924F925F926F9223
:100350007F928F929F92AF92BF92CF92DF92EF9255
:10036000FF920F931F93CF93DF93082FEB01542E2F
:10037000452E59010E94A2146B017C0110E0812CD2
:10038000912CB401600F711FC617D707A8F1C501E2
:100390000E945C1B8053E52DF42DE80FF11DE80F42
:1003A000F11D90818181382E331C3324331C692E3A
:1003B000782E31F077FE0CC071946194710808C0FA
:1003C00077FE03C071946194710888E1681A71081E
:1003D0000E94A2146C157D058E059F05C8F333207D
:1003E00011F02B9801C02B9AC60CD71CE11CF11CF4
:1003F0008FEF881A980AC5CF0E94A2146C157D054C
:100400008E059F05C8F3DF91CF911F910F91FF904B
:10041000EF90DF90CF90BF90AF909F908F907F90A4
:100420006F905F904F903F9008954F925F926F92C0
:100430007F928F929F92AF92BF92CF92DF92EF9274
:10044000FF920F931F93CF93DF93982E862E2A014E
:100450002B9A0E94A2146B017C01662457FC6094C5
:10046000762C891408F446C0692D70E081E292E090
:100470000E945C1B90ED980F9A3010F4892F01C0F8
:100480008753C4E0D0E008E0A82EBB24A7FCB094BA
:100490000E94A2146C157D058E059F05C8F310E01F
:1004A00098012A213B21232B71F02B98C40CD51CD9
:1004B000E61CF71C0E94A2146C157D058E059F0595
:1004C000C8F32B9A0DC02B9AC40CD51CE61CF71C44
:1004D0000E94A2146C157D058E059F05C8F32B980C
:1004E000C40CD51CE61CF71C15950795219781F6C1
:1004F0009394B7CF0E94A2146C157D058E059F05BD
:10050000C8F3DF91CF911F910F91FF90EF90DF9093
:10051000CF90BF90AF909F908F907F906F905F90A3
:100520004F900895CF92DF92EF92FF920F931F9317
:10053000CF93DF9300D000D000D0CDB7DEB78C01D1
:100540006B01FC01E080F1806DE071E0CE0101966D
:100550000E94CF19A701BE016F5F7F4F81E292E039
:100560000E94881B7C01CE0101960E946119FFEF59
:10057000EF16FF0601F1F801408151814F3FFFEF77
:100580005F07C9F0970161E272E0CE0101960E9417
:10059000A41BBE016F5F7F4FC6010E941B1ACE01D4
:1005A00001960E9461198FEFE81AF80AF801F182AA
:1005B000E08281E001C080E026960FB6F894DEBFAD
:1005C0000FBECDBFDF91CF911F910F91FF90EF90A4
:1005D000DF90CF900895BF92CF92DF92EF92FF927B
:1005E0000F931F93CF93DF93CDB7DEB7C856D109D2
:1005F0000FB6F894DEBF0FBECDBF67E072E0CE014C
:100600008F599F4F0E94CF196EE170E0CE018F5934
:100610009F4F0E949219A9961FAE1EAEA9970E94E5
:100620003E011FEF01E042E1F42E59E0E52E62E0C9
:10063000D62ECC24C394BE016F597F4FCE01895969
:100640009F4F0E949202882309F44FC060E070E03F
:10065000CE018F599F4F0E945C1B833589F561E065
:1006600070E0CE018F599F4F0E945C1B833419F3B9
:1006700061E070E0CE018F599F4F0E945C1B8D346A
:1006800059F41F5FE1E0F0E0EC0FFD1FF19EE00D7B
:10069000F11D1124C282CFCF61E070E0CE018F59ED
:1006A0009F4F0E945C1B823531F61F5FE1E0F0E056
:1006B000EC0FFD1FF19EE00DF11D1124D282BBCF86
:1006C00060E070E0CE018F599F4F0E945C1B803527
:1006D00009F068C062E070E0CE018F599F4F0E9420
:1006E0005C1B8D3309F05EC082C0B12C32E1C32E99
:1006F000B016D1F1D12CED2CF12CCE9CA001CF9CC9
:10070000500D1124E1E0F0E0EC0FFD1FE40FF51FA8
:100710008281823079F44A5F5F4F21E030E02C0F14
:100720003D1F420F531F6481758121E232E08381B6
:100730000E94A401CE9CF001CF9CF00D112481E019
:1007400090E08C0F9D1FE80FF91F8281813031F4FA
:1007500040815181648183810E9415022B98D3943A
:100760001D1548F6B394C4CF0E94370161E272E0D0
:1007700082E494E00E945418CE018F599F4F0E944A
:100780006119C859DF4F0FB6F894DEBF0FBECDBF59
:10079000DF91CF911F910F91FF90EF90DF90CF905D
:1007A000BF90089560E070E0CE018F599F4F0E9486
:1007B0005C1B823509F050C061E070E0CE018F59BA
:1007C0009F4F0E945C1B8D3309F046C042E050E011
:1007D000BE016F597F4FCE01855A9F4F0E942B015A
:1007E000CE01855A9F4F0E94E91B062F82C022E04E
:1007F00030E041E050E0BE016F597F4FCE01855A95
:100800009F4F0E94A41BCE01855A9F4F0E94E91B57
:10081000B62ECE01855A9F4F0E94611943E050E0E9
:10082000BE016F597F4FCE01855A9F4F0E942B0109
:10083000CE01855A9F4F0E94E91BE19EF0011124D1
:10084000EB0DF11D3396EE0FFF1F21E030E02C0F72
:100850003D1FE20FF31F4BC060E070E0CE018F59E7
:100860009F4F0E945C1B8434B9F4A9968EAD9FAD56
:10087000A997E1E0F0E0EC0FFD1FF19EE00DF11D06
:10088000112421E0280FA6963FADA697231B2383B2
:10089000029795838483CFCE60E070E0CE018F59BC
:1008A0009F4F0E945C1B833409F0C5CE61E070E06D
:1008B000CE018F599F4F0E945C1B8D3309F0BBCE38
:1008C00042E050E0BE016F597F4FCE01855A9F4FE5
:1008D0000E942B01CE01855A9F4F0E94E91BE1E047
:1008E000F0E0EC0FFD1FF19EE00DF11D112471836E
:1008F0006083CE01855A9F4F0E9461199CCE62E7AA
:1009000070E082E494E00E94061860912B0270E08F
:100910004AE050E082E494E00E941B196DE670E02A
:1009200082E494E00E9406186091290270E04AE097
:1009300050E082E494E00E941B1968E670E082E4D3
:1009400094E00E94061860912A0270E04AE050E0AC
:1009500082E494E00C942319CF93DF93CDB7DEB7F4
:10096000AE970FB6F894DEBF0FBECDBF61E070E06A
:1009700081E292E00E945C1B843729F161E070E023
:1009800081E292E00E945C1B823721F542E050E058
:1009900061E272E0CE0101960E942B0120E030E07E
:1009A00043E050E0BE01675D7F4FCE0101960E949B
:1009B0005E1BCE0101960E946119CE0189960E94AC
:1009C000F11F8093080161E272E082E494E00E94EA
:1009D000541895C061E070E081E292E00E945C1BD7
:1009E0008337F1F42B9A42E050E061E272E0CE01ED
:1009F00089960E942B0120E030E048E250E0BE01E1
:100A00006F5F7F4FCE0189960E945E1BCE01899653
:100A10000E946119CE0101960E9465012B98D3CFE7
:100A200061E070E081E292E00E945C1B8336A9F4F1
:100A300042E050E061E272E0CE0101960E942B019B
:100A4000CE0101960E94E91B709307016093060195
:100A5000CE0101960E946119B6CF61E070E081E29B
:100A600092E00E945C1B803709F049C067E072E0A9
:100A7000CE0189960E94CF1964E170E0CE0189967B
:100A80000E9492196FE071E0CE0189960E94271AA8
:100A90004AE060910801CE0101960E943F1ABE0112
:100AA0006F5F7F4FCE0189960E94C41ACE010196D6
:100AB0000E94611967E971E0CE0189960E94CB1A04
:100AC00060910601709107014AE0CE0101960E94F3
:100AD0006C1ABE016F5F7F4FCE0189960E94C41AC7
:100AE000CE0101960E946119BE01675D7F4F82E4CD
:100AF00094E00E945418CE0189960E946119AE9626
:100B00000FB6F894DEBF0FBECDBFDF91CF91089531
:100B1000CF93DF9300D0CDB7DEB72091DF043091C3
:100B2000E0042115310511F423EE34E0CE010196E5
:100B3000821B930B0F900F90DF91CF910895CF926E
:100B4000DF92EF92FF920E9496146B017C0128EED7
:100B500033E040E050E00E94D81D8091180290914F
:100B60001902A0911A02B0911B02C816D906EA0612
:100B7000FB0648F48091160290911702019690931B
:100B8000170280931602C0921802D0921902E092C6
:100B90001A02F0921B02CA01B901FF90EF90DF9098
:100BA000CF9008956AE171E082E494E00E946618B3
:100BB00061E070E080E090E00C94C51461E070E0CA
:100BC00081E292E00E945C1B813511F40E943E019B
:100BD00061E070E081E292E00E945C1B853411F4D8
:100BE0000C9437010895262F220F330B94E049020D
:100BF000B0011124682B622B81E090E00C94D52287
:100C0000CF93DF9361E070E081E292E00E945C1B91
:100C1000873421F4DF91CF910C947F0462E070E07F
:100C200081E292E00E945C1B833599F062E070E003
:100C300081E292E00E945C1B853571F062E070E019
:100C400081E292E00E945C1B833441F4CAE2D2E06C
:100C500005C0CBE2D2E002C0C9E2D2E061E070E0C0
:100C600081E292E00E945C1B853419F481E0888364
:100C700009C061E070E081E292E00E945C1B843474
:100C800059F4188240912A026091290280912B0226
:100C9000DF91CF910C94F305DF91CF91089560E03F
:100CA00070E081E292E00E945C1B803511F40C94AC
:100CB000D20560E070E081E292E00E945C1B8F331D
:100CC00009F072C06FE382E494E00E9437186AE88A
:100CD00070E082E494E00E94061866E582E494E005
:100CE0000E94371860E282E494E00E94371869E6B7
:100CF00082E494E00E94371860E282E494E00E946B
:100D0000371862E582E494E00E94371860E282E4DA
:100D100094E00E94371864E782E494E00E94371858
:100D200060E282E494E00E94371868E582E494E08F
:100D30000E94371860E282E494E00E94371866E46B
:100D400082E494E00E94371860E282E494E00E941A
:100D5000371863E582E494E00E94371860E282E489
:100D600094E00E94371860E582E494E00E9437180E
:100D700060E282E494E00E94371863E482E494E045
:100D80000E94371860E282E494E00E94371867E41A
:100D900082E494E00E94371860E282E494E00E94CA
:100DA000371867E072E00AC060E070E081E292E02C
:100DB0000E945C1B863531F46DE171E082E494E0C1
:100DC0000C94661860E070E081E292E00E945C1B87
:100DD000823549F40E9488054AE050E0BC0182E473
:100DE00094E00C94231960E070E081E292E00E94AC
:100DF0005C1B893641F488E292E00E94E508892B69
:100E000081F40C94AC0460E070E081E292E00E9416
:100E10005C1B833561F488E292E00E94E508892B2F
:100E200021F081E080931C0208950C94EB0260E0B5
:100E300070E081E292E00E945C1B843751F40E94D2
:100E40009F05AB01BC012AE030E082E494E00C9401
:100E50004F1960E070E081E292E00E945C1B8835EF
:100E600011F40C94DE0560E070E081E292E00E94F3
:100E70005C1B8634D1F060E070E081E292E00E9479
:100E80005C1B833411F40C94000660E070E081E296
:100E900092E00E945C1B873411F40C947F0466E797
:100EA00070E082E494E00C94421808951F93CF936D
:100EB000DF9300D0CDB7DEB780911C02882389F084
:100EC00010921C020E944F0680911C02811106C0E4
:100ED00067E072E081E292E00E94271A81E080934D
:100EE000270211E080916303882341F1809163031D
:100EF00081508093630380916503609162030E9437
:100F0000A41D90936503E091650381E08E0F8093AB
:100F10006503F0E0EE0FFF1FEA59FC4F80819181DD
:100F20009A838983BE016F5F7F4F88E292E00E94BF
:100F3000AA138823B9F210932702D4CF0F900F90F1
:100F4000DF91CF911F910895EF92FF920F931F931E
:100F5000CF93DF93EC017B018A0181E090E00E9456
:100F6000CD22982F9170988381FB992790F9F701F2
:100F7000908382FB882780F9F8018083DF91CF91ED
:100F80001F910F91FF90EF90089526E040E051EE01
:100F900060E070E082E494E00E94AE1660E082E0DF
:100FA0000E945C1561E08BE00E945C1561E08DE0C1
:100FB0000E945C1580E1809381001092800082E0A5
:100FC0008093FE0388E199E7909300048093FF03E8
:100FD000909387008093860082E1809381008CEF5C
:100FE00090E09093FD038093FC0381E080936F0079
:100FF00080E090E00E94CD228B3049F44AE252E03A
:1010000069E272E08BE292E00E94A4070AC06BE002
:1010100080E090E00E94D52267E081E090E00E94AD
:10102000D5220E94370164E170E081E292E00C94E5
:1010300092190F931F93CF93DF938BE480936203F6
:10104000109263031092650310926403CBE3D3E024
:10105000D0934003C0933F030DE313E0109342038A
:101060000093410367E072E085E593E00E94CF19A9
:1010700067E072E08BE593E00E94CF19F8011182DE
:1010800010821982188288E292E00E94A70867E025
:1010900072E081E292E00E94CF190E94A214609354
:1010A0001D0270931E0280931F0290932002DF9115
:1010B000CF911F910F9108950C941F01CF93C1E020
:1010C00082E494E00E94CB15892BB9F082E494E08D
:1010D0000E94E4158A3041F01CF4882329F007C0EF
:1010E0008D3011F0833219F4C0931C02E9CF682FC0
:1010F00081E292E00E94DB1AE3CFCF9108951F9224
:101100000F920FB60F9211242F933F934F935F933B
:101110006F937F938F939F93AF93BF93EF93FF93BF
:10112000E091FC03F091FD030995FF91EF91BF91D0
:10113000AF919F918F917F916F915F914F913F916F
:101140002F910F900FBE0F901F9018950895FC01DE
:10115000E85FFE4F1082B39610827B971082319623
:10116000118210827B962FEF2083FC012083AC013B
:1011700020E030E0FA01E15EFE4F11821082FC01B6
:10118000E20FF31F14822F5F3F4F4E5F5F4F2630F9
:10119000310581F7FC01E55FFE4F1082339626E9A9
:1011A00030E0318320833D964DEC5CEC6CE47EE3D3
:1011B00040835183628373837297108233961082C7
:1011C0003196108233971082089580E090E0089560
:1011D000CF93DF93FC01E55DFE4FD081C0E07D97AA
:1011E000CD17C1F0DC01A15EBE4F2D913C91AB014A
:1011F000421B530B9A0157FF03C0319521953109CA
:101200000296408151814217530714F08C2F03C07E
:10121000CF5FE6CF8FEFDF91CF910895FC0114826D
:1012200015821682178210861186411104C0DC01D6
:10123000A85FBE4F4C91641780F4DF01A60FB11D6B
:101240001A968C91DF01A80FB11D14968C911497FA
:101250008F5F14968C936F5FEECF08952F923F921D
:101260004F925F926F927F928F929F92AF92BF92B6
:10127000CF92DF92EF92FF920F931F93CF93DF9362
:10128000CDB7DEB72E970FB6F894DEBF0FBECDBF39
:101290009E878D8740E060E00E940E09ED85FE8507
:1012A000E55DFE4F5080712C2D853E85255E3E4FBD
:1012B0003A8729878D859E85885F9E4F9C878B877F
:1012C000751409F4C3C044244394470C642C272CA0
:1012D000312CC101880F991FAD85BE858A0F9B1FD8
:1012E000FC01E15EFE4FFA83E9832A0E3B1EF4E027
:1012F0002F0E311C29813A8138872F83651409F418
:10130000A3C0862D90E09C838B83880F991F9E83BA
:101310008D83FC01AD85BE85EA0FFB1FE15EFE4FAC
:1013200000811181C80117FF04C088279927801BFD
:10133000910BBC01882777FD8095982F0E948D1C0A
:10134000E985FA8520813181428153810E94411DC6
:101350004B015C01A981BA81CD90DC907801EC1839
:10136000FD08F7FE03C0F194E194F10820E030E0BD
:1013700040E05FE3C501B4010E94411D9B01AC0147
:10138000C501B4010E94F61B0E945A1C6E157F0510
:101390000CF458C0EB85FC85208180E090E082173A
:1013A00050F4ED85FE85E80FF91F3285361101C036
:1013B00072860196F4CFD1014C91552747FD509587
:1013C000EB81FC812D853E85E20FF31FE481FF2731
:1013D000E7FDF0959A012E0F3F1F21153105E1F42D
:1013E000C49EC001C59E900DD49E900D1124B901DC
:1013F0000E94C41D7B010E9FC0010F9F900D1E9F78
:10140000900D1124B9010E94C41DE60EF71EAF8194
:10141000B885ED92FC920CC00C0D1D1D17FF02C08B
:101420000F5F1F4F15950795E981FA81118300839E
:10143000ED81FE812D853E85E20FF31FE15EFE4FBB
:101440001182108263945ACF742C3ACF2E960FB625
:10145000F894DEBF0FBECDBFDF91CF911F910F91EA
:10146000FF90EF90DF90CF90BF90AF909F908F90C4
:101470007F906F905F904F903F902F9008953F9294
:101480004F925F926F927F928F929F92AF92BF9294
:10149000CF92DF92EF92FF920F931F93CF93DF9340
:1014A000EC018FEF8883FE01E55DFE4F30806E0119
:1014B00000E010E0EE24EA94FE2C4E0188EF881A3A
:1014C0008EEF980A031508F06AC0F601E15EFE4F40
:1014D0005F01FFEFEF16FF0639F5F501808191817D
:1014E00097FD22C0FE01E00FF11F6481772767FDA1
:1014F0007095872F972F0E948D1C2B013C01F401C2
:10150000608170E080E090E00E948D1C2BE734E168
:101510004EE25EE30E94411D9B01AC01C301B2019A
:101520000E943D1D1816A4F1F5012081318137FD7F
:1015300030C0C701880F991F8C0F9D1FFC01E15E11
:10154000FE4F80819181281739071CF5FE01E00FBD
:10155000F11F6481772767FD7095872F972F0E9471
:101560008D1C2B013C01F401608170E080E090E073
:101570000E948D1C2BE734E14EE25EE30E94411D88
:101580009B01AC01C301B2010E943D1D18160CF471
:1015900078010F5F1F4FF2E0CF0ED11C93CF8FEF7A
:1015A000E816F80641F0E882CF5EDE4F81E090E079
:1015B0009983888301C080E0DF91CF911F910F91C3
:1015C000FF90EF90DF90CF90BF90AF909F908F9063
:1015D0007F906F905F904F903F9008958F929F9271
:1015E000AF92BF92CF92DF92EF92FF920F931F9331
:1015F000CF93DF93FC018C010F5E1E4FD8018D91BC
:101600009C911197019709F07CC05A96BC90BA94AE
:10161000C7E0AC2E6F01B8EFCB1ABEEFDB0AB7FC08
:1016200070C02B2D332727FD3095C901880F991FD6
:101630008E0F9F1FDC01A15EBE4FCD91DC91D7FFC5
:101640005EC0D195C195D109C83682E4D80708F0AB
:1016500056C0E080FF24E7FCF094C701880F991F73
:101660008E0F9F1FDC01A15EBE4F8D909C90CE011E
:10167000B4010E94B01D6832710508F040C0A89CFA
:10168000C001A99C900D11248C179D07C0F5DF01A6
:10169000A20FB31F14968C9186308CF5D6014C9115
:1016A00050E0BA0161507109912C892D90E08617A4
:1016B000970784F4DF01A80FB91F1B96CC911B97E5
:1016C000D0E0C217D307C9F41A96AC91B0E0AE15BA
:1016D000BF0599F4485251098417950784F4DF0136
:1016E000A45DBE4FBC9282E090E0D8018D939C93A4
:1016F000E75FFE4F908281E009C09394D6CFBA9401
:101700008ECFE45DFE4F8FEF808380E0DF91CF913D
:101710001F910F91FF90EF90DF90CF90BF90AF900F
:101720009F908F9008950F931F93CF93DF938A011B
:10173000E90182E494E00E942918B80182E494E06F
:101740000E942918BE0182E494E0DF91CF911F919D
:101750000F910C942918EF92FF920F931F93CF9340
:10176000DF93EC01F62EE42EB90182E494E00E94AE
:101770002918EF1460F0FE01EF0DF11D4AE050E072
:10178000628582E494E00E944819F394F2CFB80194
:1017900082E494E00E94291880E0DF91CF911F91AC
:1017A0000F91FF90EF90089570E0FC0126A1332780
:1017B00027FD30956217730751F027A1332727FDC6
:1017C000309581E06217730719F080E0089581E099
:1017D000089570E0FC0120A5332727FD309562179E
:1017E000730751F021A5332727FD309581E062175B
:1017F000730719F080E0089581E008959F92AF92F9
:10180000BF92CF92DF92EF92FF920F931F93CF93ED
:10181000DF9300D01F92CDB7DEB78C017B0120E3B0
:1018200030E340E029833A834B83FC01668DF3E08B
:101830006F9FB0011124C7010E949219E114F104B5
:1018400049F1912C87ECA82E81E0B82ECE010196AB
:101850006C01F801868D8915E8F0F80183A19816CE
:1018600020F4E90DF11D808101C08FEF1F928F934D
:10187000BF92AF92DF92CF920E94D920B601C701EA
:101880000E94CB1A93940F900F900F900F900F908F
:101890000F90DFCF0F900F900F90DF91CF911F919E
:1018A0000F91FF90EF90DF90CF90BF90AF909F90FF
:1018B00008950F931F93CF93DF938C01EB0160E2A8
:1018C00070E0CE010E949219209709F468C06CEC78
:1018D00071E0CE010E94CB1AF80184A195A126A146
:1018E000220F330B820F931FFC01E15EFE4F6081DC
:1018F0007181CE010E941A1B6BE3CE010E94DB1A9C
:1019000060ED71E0CE010E94CB1AF80184A195A18F
:1019100027A1220F330B820F931FFC01E15EFE4FC4
:1019200060817181CE010E941A1B6BE3CE010E947F
:10193000DB1A64ED71E0CE010E94CB1AF80184A19C
:1019400095A120A5220F330B820F931FFC01E15EAE
:10195000FE4F60817181CE010E941A1B6BE3CE01A4
:101960000E94DB1A68ED71E0CE010E94CB1AF801EB
:1019700084A195A121A5220F330B820F931FFC0197
:10198000E15EFE4F60817181CE010E941A1B6BE304
:10199000CE01DF91CF911F910F910C94DB1ADF9153
:1019A000CF911F910F9108950F931F93CF93DF93C2
:1019B0008C01EB0167E070E0CE010E949219209744
:1019C00099F06CED71E0CE010E94CB1AF80162A58E
:1019D00073A5CE010E941A1B6BE3CE01DF91CF915C
:1019E0001F910F910C94DB1ADF91CF911F910F91F2
:1019F00008954F925F926F927F928F929F92AF92D3
:101A0000BF92CF92DF92EF92FF920F931F93CF93EB
:101A1000DF93EC010CA11DA1580185EDA81A8EEFF2
:101A2000B80AF5018081843008F4C4C06801F8EF79
:101A3000CF1AFEEFDF0AF601608170E080E090E0EF
:101A40000E948D1C2AE037ED43E25DE30E94411DB8
:101A50000E945F1C40E050E0912C812CEE24EA941F
:101A6000FE2C262F30E0F5018081481708F06BC06E
:101A7000642F70E0F801E60FF71FE4818E2F99279D
:101A800087FD9095821793070CF45BC0660F771F54
:101A9000600F711FDB01A15EBE4F6D917C91161628
:101AA00017064CF55E0F8394E60EF71EEFA1EF3F8D
:101AB00069F08E2F880F990B800F911FDC01A15EBA
:101AC000BE4F8D919C91861797070CF4E42FEFA3DE
:101AD000E9A5EF3F69F08E2F880F990B800F911FBA
:101AE000DC01A15EBE4F8D919C91681779070CF4C3
:101AF000E42FE9A726C05E1B9394EEA1EF3F69F0A7
:101B00008E2F880F990B800F911FDC01A15EBE4FB5
:101B10008D919C91681779070CF4E42FEEA3E8A54A
:101B2000EF3F69F08E2F880F990B800F911FDC011A
:101B3000A15EBE4F8D919C91861797070CF4E42F00
:101B4000E8A74F5F90CF652F70E080E090E00E94A3
:101B50008D1C2B013C01F601608170E080E090E07B
:101B60000E948D1C2AE037ED43EA5CE30E94411D90
:101B70009B01AC01C301B2010E943D1D1816D4F0B7
:101B8000981018C0C70163E070E00E94C41D7BA7D5
:101B90006AA79EA19F3F71F088A58F3F59F09817C3
:101BA00049F02FA12F3F31F099A59F3F19F081E017
:101BB000291301C080E0DF91CF911F910F91FF9019
:101BC000EF90DF90CF90BF90AF909F908F907F90DD
:101BD0006F905F904F900895FC0183A12E2FDF013D
:101BE0009A2F921B981710F41D92FACF168E178E0B
:101BF00087E082A3089524E1FC0124A70C94EC0D56
:101C00007F928F929F92AF92BF92CF92DF92EF928C
:101C1000FF920F931F93CF93DF93EC018CA19DA1B3
:101C2000FC01E45FFE4F108233971082812CBB24AD
:101C3000B39437E0A32E0CA11DA1F801E85FFE4F7D
:101C40008081881608F0A3C08DA5811110C0F8010D
:101C5000E80DF11DF2846F2DCE010E94D40B81118D
:101C6000DFC06F2DCE010E94E90B8111D9C0CDA438
:101C70000CA11DA1CC2079F18EA581112CC0C80129
:101C8000885F9E4F7C01F801E80DF11DD2846D2D17
:101C9000CE010E94D40B811105C0F7018081881606
:101CA00008F4C8C0282DF70180818816A0F4C80167
:101CB0008D0D911D8D0D911DFC01E15EFE4F9180FA
:101CC000991C9924991CF801E75FFE4F8080281920
:101CD00009F0ACC0BEA68EA5882309F456C0CC205E
:101CE00009F453C0E82CF12C6801CE0CDF1CF6017E
:101CF0007284672DCE010E94D40B882311F09B249F
:101D00001CC0672DCE010E94E90B782E882309F4B0
:101D100093C0F801E85FFE4F208130E02150310987
:101D2000E216F3060CF088C0F6016385CE010E942E
:101D3000E90B882309F480C083944E8D8BA148174A
:101D400020F55AA1852F90E0292D332727FD3095C6
:101D5000052E01C0220F0A94EAF7FE01E40FF11DDF
:101D60003081322B30832F8D2F5F2F8F28A1821B44
:101D7000910997FD03C0521B5AA307C0AAA24F5F47
:101D80004E8FFE01E40FF11D1082839454CF881210
:101D90003AC0D801A75FBE4F4C91423058F12F8D09
:101DA00030E08CA587FD8F5F8595992787FD9095FD
:101DB0008217930744F5841A80828CA19DA1FC01AF
:101DC000E85FFE4F408150E04F5F5F4F319660818A
:101DD00070E0665F7F4F680F791F0A960E943F2070
:101DE0008CA19DA1FC01E45FFE4F21E02083BD9604
:101DF000208314C0411107C0D801A75CBE4F81E009
:101E00008C9310820BC04F8D50E02CA5332727FDFB
:101E1000309581E0421753070CF071C080E06FC02D
:101E2000F801E75FFE4F8082BDA621CF20FF52CF91
:101E3000839450CF839427CF4F8D50E02CA5332728
:101E400027FD309542175307CCF4772089F0F8012D
:101E5000E85FFE4F808190E00197E816F90644F4B0
:101E6000F6016385CE010E94E90B882309F442C084
:101E70001DA61EA6CE010E94EC0D5FCFF801E65F05
:101E8000FE4F80828CA19DA1FC01E85FFE4FDC012A
:101E9000A65FBE4F20818C91281B20838CA19DA121
:101EA000FC01E85FFE4F408150E04F5F5F4F32968C
:101EB000608170E0665F7F4F680F791F0A960E940D
:101EC0003F200CA11DA1F801E45FFE4FFF24F39415
:101ED000F08234978081F801E80FF11D6285CE0110
:101EE0000E94E90B882309F48ECFF801E75CFE4FCE
:101EF000F08294CFF801E75FFE4F8080B9CFDF9189
:101F0000CF911F910F91FF90EF90DF90CF90BF90F6
:101F1000AF909F908F907F9008953F924F925F92E5
:101F20006F927F928F929F92AF92BF92CF92DF92E9
:101F3000EF92FF920F931F93CF93DF9300D000D0C7
:101F400000D0CDB7DEB77C015C0187ECA81A8EEF1C
:101F5000B80AF5018081811105C0F197808188322E
:101F600008F4B4C2C7010E942E0940E060E0C70136
:101F70000E940E09C7010E943F0AC7010E94EE0A93
:101F8000F7018381882309F42BC1EF5EFE4F808126
:101F90009181029709F024C14701F7EF8F1AFEEFF4
:101FA0009F0AF40160815701F6EFAF1AFEEFBF0AF6
:101FB00082E0860FF50180838701085F1E4FF801DC
:101FC0007081872F90E00197D701A45DBE4FF50186
:101FD000D0802D2D30E0281739070CF5F701E20FDE
:101FE000F31F438550E02C91332727FD309542178E
:101FF000530781F4428550E0F7012081332727FD04
:1020000030954217530731F4DA94F501D082DD247C
:10201000D39406C0D394D394F501D082D8CFD12CD9
:10202000F5018081781708F47083F5014081C701BC
:102030000E940E09DD2051F0F501808190E0F4014D
:102040002081821B9109889734F4C6C0F801408131
:102050004E3F08F0A2C06701F3EDCF1AFEEFDF0A92
:1020600067E072E0C6010E94271A87010D5C1E4FCF
:1020700067E072E0C8010E94271A62E0C6010E9470
:10208000DB1A6FED71E0C6010E94CB1A6BE3C6014B
:102090000E94DB1A312C370185ED681A8EEF780A21
:1020A000F3018081381640F5432C512CF701E40DE3
:1020B000F51D84818823F1F060E5C6010E94DB1ADA
:1020C000632DC6010E94EE1A6DED71E0C6010E94FB
:1020D000CB1AC201880F991F8E0D9F1DFC01E15E76
:1020E000FE4F60817181C6010E941A1B6BE3C6011D
:1020F0000E94DB1A3394D4CF62EE71E0C6010E94D5
:10210000CB1A6BE3C8010E94DB1A65EE71E0C801CF
:102110000E94CB1AF7016081772767FD7095C8018F
:102120000E941A1B6BE3C8010E94DB1A69EE71E082
:10213000C8010E94CB1AF701E45DFE4F608177274A
:1021400067FD7095C8010E941A1B6BE3C8010E94CD
:10215000DB1AF701E35FFE4F8081882349F06DEEC3
:1021600071E0C8010E94CB1A6BE3C8010E94DB1A20
:1021700063E0C8010E94DB1A6AE0C8010E94DB1A12
:102180009601F5014081F4016081C7010E94AB0B0B
:1021900081E0F701E55FFE4F1DC0F4016081623010
:1021A000D8F0F501808190E08D3F9105ACF0461BA1
:1021B000F801408350E04F5F5F4F70E0665F7F4FF4
:1021C0006E0D7F1DC7010A960E943F2081E0F70136
:1021D000E45FFE4F80832AC1C7010E94A70826C181
:1021E000F7018181811104C08281882309F41AC119
:1021F000F701EF5EFE4F80819181019709F012C1D6
:102200004701F8EF8F1AFEEF9F0AF40180818832B0
:1022100008F408C16701F3EDCF1AFEEFDF0A67E0AB
:1022200072E0C6010E94271A87010D5C1E4F67E00D
:1022300072E0C8010E94271A62E0C6010E94DB1A00
:10224000F7018281882309F463C0809131048111F0
:1022500043C08EE18093240481E080932104109296
:10226000220481E094E00E94EC0D2091210487E09B
:1022700090E0821B91097091220467E041E050E0F8
:10228000262F30E0821793074CF49A01062E01C0E6
:10229000220F0A94EAF7722B6150F2CF7093220456
:1022A0008FEF8093270480932804809329048093E0
:1022B0002A0410922E0410922F04F0922604E09229
:1022C000250481E094E00E94FB0D81E080933104BD
:1022D00086EA98E00E94B517F5018081811107C058
:1022E00081E094E00E94FB0D81E180932D04F501D3
:1022F0008081882339F081E094E00E94000E8111F2
:102300009FC006C081E094E00E94F90C8111F3CFD8
:10231000F7018181882309F489C05701F5EFAF1ACD
:10232000FEEFBF0AF5018081811180C06FEE71E080
:10233000C6010E94CB1A6BE3C6010E94DB1A312C46
:102340003701F5ED6F1AFEEF7F0AF3018081381631
:1023500048F5432C512CF701E40DF51D84818823A9
:10236000F9F060EC71E0C6010E94CB1A632DC60142
:102370000E94EE1A6DED71E0C6010E94CB1AC201F7
:10238000880F991F8E0D9F1DFC01E15EFE4F60813D
:102390007181C6010E941A1B6BE3C6010E94DB1A01
:1023A0003394D3CF62EE71E0C6010E94CB1A6BE387
:1023B000C8010E94DB1A65EE71E0C8010E94CB1AC9
:1023C000F7016081772767FD7095C8010E941A1B8D
:1023D0006BE3C8010E94DB1AF701E35FFE4F8081C7
:1023E000882349F06DEE71E0C8010E94CB1A6BE3BF
:1023F000C8010E94DB1A63E0C8010E94DB1A6AE090
:10240000C8010E94DB1AF40140814150960160E04E
:10241000C7010E94AB0BF701E45FFE4F108281E021
:10242000F501D8CEF701E55FFE4F1082F701E45FBA
:10243000FE4F808181114AC0C7010E94A70846C093
:1024400067E072E0CE0101960E94CF1962EE71E062
:10245000CE0101960E94271ABE016F5F7F4F81E077
:1024600094E00E94FE0B62EF71E0C6010E94CB1A5D
:102470006BE3C6010E94DB1AB60181E094E00E9482
:10248000590C6BE3C8010E94DB1AB80181E094E0AB
:102490000E94D40C63E0C8010E94DB1A6AE0C80104
:1024A0000E94DB1A9801AE014F5F5F4FB601C70172
:1024B0000E94930BF501108281E0F701E55FFE4F6A
:1024C0008083CE0101960E94611922CF26960FB615
:1024D000F894DEBF0FBECDBFDF91CF911F910F915A
:1024E000FF90EF90DF90CF90BF90AF909F908F9034
:1024F0007F906F905F904F903F9008958F929F9242
:10250000AF92BF92CF92DF92EF92FF920F931F9301
:10251000CF93DF931F92CDB7DEB74C018C01085FDC
:102520001E4FD8018C9190E08D3F910544F081E0E1
:10253000F401E35FFE4F8083C4010E948D0FF4011C
:10254000E05FFE4F10826401B9EECB1ABEEFDB0AEA
:10255000D601ED91FC9111978081918112960D9099
:10256000BC91A02D2D913C91D8014C9150913004FB
:102570007401B5EDEB1ABEEFFB0AD7016C9165173C
:1025800008F45C93442361F082279327B92EBB1C87
:10259000BB24BB1C81E04D3F09F480E0B82205C09C
:1025A000D7011C9210923004B12C60817181C4015A
:1025B00049830E94E808A82E498187FD2CC0F401B8
:1025C000E40FF11D8287423030F081858A1103C00B
:1025D000C4010E94A7088A2D880F990B880D991DA8
:1025E000FC01E15EFE4FD6018D919C9120813181ED
:1025F000DC018D919C91280F391F37FF02C02F5F9E
:102600003F4F3595279531832083F80180818F5F77
:10261000808320E012C040E060E0C4010E940E0907
:10262000D7018C91863041F480913004F401E80F99
:10263000F11D8481823024F421E0B1101DC001C05D
:1026400020E0F8018081A401455F5E4F5A01883285
:1026500048F081E0DA018C93C4010E948D0F109242
:1026600030046AC0C40129830E94A708F5011082C2
:102670001092300429810BC0D8018C91883238F037
:1026800083E090E0F401EF5EFE4F9183808322238C
:1026900009F452C0F80140815091300480E090E08C
:1026A000242F30E0F9013197280D391DBF01680F43
:1026B000791F6F3FAFEF7A07E1F00197D901A80FBB
:1026C000B91F1A96AC91A513F1CFCB010196481B07
:1026D000D8014C9350E04F5F5F4F655F7F4F680DAF
:1026E000791DC4010A960E943F20F80180818F5F06
:1026F000808340913004D601ED91FC91208131819D
:10270000C401840F911D840F911DFC01E15EFE4FF9
:1027100031832083F8018081F401E80FF11D4287A5
:102720008F5FD8018C934F5F40933004463021F483
:1027300010923004F70140830F90DF91CF911F91E9
:102740000F91FF90EF90DF90CF90BF90AF909F9050
:102750008F900895CF93DF93EC01C55FDE4F188211
:10276000FC01E75EFE4F0190F081E02D2081318178
:10277000DC01A95EBE4F0D90BC91A02D2D933C9322
:10278000DB012D913C91318320830E947E12888150
:10279000DF91CF91089508958230E8F4E82FF0E0BA
:1027A000EE0FFF1FE75FFE4F71836083813041F0C2
:1027B000809169008C7F842B80936900E89A08954A
:1027C00080916900440F551F440F551F837F842B50
:1027D00080936900E99A0895823078F4813011F08D
:1027E000E89801C0E998E82FF0E0EE0FFF1FE75FDF
:1027F000FE4F8BEC93E19183808308951F920F929B
:102800000FB60F9211242F933F934F935F936F93C3
:102810007F938F939F93AF93BF93EF93FF93E09139
:102820000901F0910A010995FF91EF91BF91AF91D4
:102830009F918F917F916F915F914F913F912F91D8
:102840000F900FBE0F901F9018951F920F920FB60A
:102850000F9211242F933F934F935F936F937F9326
:102860008F939F93AF93BF93EF93FF93E0910B01EF
:10287000F0910C010995FF91EF91BF91AF919F915C
:102880008F917F916F915F914F913F912F910F9019
:102890000FBE0F901F9018951F920F920FB60F92B8
:1028A00011242F933F938F939F93AF93BF93809166
:1028B0003A0490913B04A0913C04B0913D043091C6
:1028C000390423E0230F2D3720F40196A11DB11DFB
:1028D00005C026E8230F0296A11DB11D20933904DF
:1028E00080933A0490933B04A0933C04B0933D043E
:1028F00080913E0490913F04A0914004B091410426
:102900000196A11DB11D80933E0490933F04A093B6
:102910004004B0934104BF91AF919F918F913F913B
:102920002F910F900FBE0F901F9018952FB7F8940E
:1029300060913A0470913B0480913C0490913D0475
:102940002FBF08953FB7F89480913E0490913F04C3
:10295000A0914004B091410426B5A89B05C02F3F2B
:1029600019F00196A11DB11D3FBF6627782F892F51
:102970009A2F620F711D811D911D42E0660F771F16
:10298000881F991F4A95D1F70895CF92DF92EF9251
:10299000FF92CF93DF936B017C010E94A214EB01A5
:1029A000C114D104E104F10489F00E94F41B0E94D7
:1029B000A2146C1B7D0B683E734090F381E0C81A33
:1029C000D108E108F108C851DC4FEACFDF91CF917F
:1029D000FF90EF90DF90CF9008958230910538F00E
:1029E000880F991F880F991F05970197F1F7089590
:1029F000789484B5826084BD84B5816084BD85B5DA
:102A0000826085BD85B5816085BDEEE6F0E08081A0
:102A100081608083E1E8F0E01082808182608083C1
:102A2000808181608083E0E8F0E080818160808344
:102A3000E1EBF0E0808184608083E0EBF0E0808176
:102A400081608083EAE7F0E0808184608083808118
:102A500082608083808181608083808180688083C0
:102A60001092C1000895833081F028F4813099F0EC
:102A70008230A1F008958730A9F08830B9F0843011
:102A8000D1F4809180008F7D03C0809180008F778A
:102A900080938000089584B58F7702C084B58F7DC0
:102AA00084BD08958091B0008F7703C08091B000FD
:102AB0008F7D8093B0000895CF93DF9390E0FC0169
:102AC000E555FF4F2491FC01E154FF4F8491882389
:102AD00049F190E0880F991FFC01E352FF4FA59147
:102AE000B4918D529F4FFC01C591D4919FB7611154
:102AF00008C0F8948C91209582238C93888182233E
:102B00000AC0623051F4F8948C91322F30958323AF
:102B10008C938881822B888304C0F8948C91822BBB
:102B20008C939FBFDF91CF9108950F931F93CF9305
:102B3000DF931F92CDB7DEB7282F30E0F901E956B9
:102B4000FF4F8491F901E555FF4F1491F901E154CC
:102B5000FF4F04910023C9F0882321F069830E946C
:102B600033156981E02FF0E0EE0FFF1FED52FF4FAC
:102B7000A591B4919FB7F8948C91611103C0109501
:102B8000812301C0812B8C939FBF0F90DF91CF9148
:102B90001F910F910895FC01818D228D90E0805C42
:102BA0009F4F821B91098F7399270895FC01918D86
:102BB000828D981731F0828DE80FF11D858D90E0A0
:102BC00008958FEF9FEF0895FC01918D828D9817E6
:102BD00061F0828DDF01A80FB11D5D968C91928D01
:102BE0009F5F9F73928F90E008958FEF9FEF0895FE
:102BF00088E697E1892B49F08EE598E0892B29F04A
:102C00000E94681781110C945E080895FC01848D60
:102C1000DF01A80FB11DA35ABF4F2C91848D90E006
:102C200001968F739927848FA689B7892C93A089E1
:102C3000B1898C9180648C93938D848D981306C098
:102C40000288F389E02D80818F7D80830895CF9362
:102C5000DF93EC01888D8823C9F0EA89FB898081A4
:102C600085FD05C0A889B9898C9186FD0FC00FB676
:102C700007FCF5CF808185FFF2CFA889B9898C91B7
:102C800085FFEDCFCE010E940616E7CFDF91CF91F1
:102C90000895CF92DF92FF920F931F93CF93DF930C
:102CA0001F92CDB7DEB76C0181E0D60158968C93A8
:102CB00058975B969C915B975C968C915C97981368
:102CC00007C05096ED91FC915197808185FD2EC0F3
:102CD000F601038D10E00F5F1F4F0F731127F02EC9
:102CE000F601848DF81211C00FB607FCF9CFD6019A
:102CF0005096ED91FC915197808185FFF1CFC601EF
:102D000069830E9406166981EBCF838DE80FF11D60
:102D1000E35AFF4F6083D6015B960C935B97529604
:102D2000ED91FC915397808180620CC0D60156963C
:102D3000ED91FC91579760835096ED91FC915197DE
:102D400080818064808381E090E00F90DF91CF915B
:102D50001F910F91FF90DF90CF900895BF92CF9277
:102D6000DF92EF92FF92CF93DF93EC016A017B0138
:102D7000B22EE889F98982E08083411581EE5807F7
:102D800061057105A1F060E079E08DE390E0A701B5
:102D900096010E94D81D21503109410951095695CB
:102DA000479537952795211580E1380798F0E889F0
:102DB000F989108260E874E88EE190E0A70196013D
:102DC0000E94D81D21503109410951095695479556
:102DD00037952795EC85FD853083EE85FF8520832B
:102DE000188EEC89FD89B082EA89FB898081806137
:102DF0008083EA89FB89808188608083EA89FB89F6
:102E0000808180688083EA89FB8980818F7D8083CF
:102E1000DF91CF91FF90EF90DF90CF90BF9008951A
:102E20001F920F920FB60F9211242F938F939F939F
:102E3000EF93FF93E0915204F09153048081E0916D
:102E40005804F091590482FD12C0908180915B0476
:102E50008F5F8F7320915C04821751F0E0915B04C7
:102E6000F0E0EE5BFB4F958F80935B0401C08081A7
:102E7000FF91EF919F918F912F910F900FBE0F9027
:102E80001F9018951F920F920FB60F9211242F9337
:102E90003F934F935F936F937F938F939F93AF93E2
:102EA000BF93EF93FF9382E494E00E940616FF9194
:102EB000EF91BF91AF919F918F917F916F915F91B2
:102EC0004F913F912F910F900FBE0F901F9018952B
:102ED00082E494E00E94CB1521E0892B09F420E0E4
:102EE000822F0895109245041092440488EE93E0D6
:102EF000A0E0B0E08093460490934704A093480478
:102F0000B093490489EF91E0909343048093420485
:102F100085EC90E090934F0480934E0484EC90E015
:102F2000909351048093500480EC90E0909353046C
:102F30008093520481EC90E0909355048093540464
:102F400082EC90E0909357048093560486EC90E0D6
:102F5000909359048093580410925B0410925C047F
:102F600010925D0410925E04089580E090E0089550
:102F700008950E94F8140E94B8170E94C507C8EF70
:102F8000D5E10E9456072097E1F30E94F815F9CF8A
:102F9000CF92DF92EF92FF920F931F93CF93DF9325
:102FA0007C016A01EB0100E010E00C151D0571F0D9
:102FB0006991D701ED91FC910190F081E02DC7015D
:102FC0000995892B19F00F5F1F4FEFCFC801DF91D3
:102FD000CF911F910F91FF90EF90DF90CF900895C8
:102FE0006115710581F0DB010D900020E9F7AD015D
:102FF00041505109461B570BDC01ED91FC910280B9
:10300000F381E02D099480E090E00895EF92FF9223
:103010000F931F93CF93DF938C017B01C0E0D0E02F
:10302000F701EC0FFD1F6491662359F0F801A081B0
:10303000B181ED91FC91C8010995892B11F0219680
:10304000EFCFCE01DF91CF911F910F91FF90EF90C5
:103050000895DC01ED91FC91DB0114964D915C919A
:1030600015976D917C910280F381E02D0994DC012C
:10307000ED91FC910190F081E02D099465E072E002
:103080000C94F0170F931F93CF93DF93EC010E94E2
:1030900006188C01CE010E943E18800F911FDF910F
:1030A000CF911F910F9108950F931F93CF93DF93AB
:1030B000EC010E9429188C01CE010E943E18800F5D
:1030C000911FDF91CF911F910F9108950F931F933F
:1030D000CF93DF93EC010E94F0178C01CE010E9488
:1030E0003E18800F911FDF91CF911F910F9108958E
:1030F0008F929F92AF92BF92CF92DF92EF92FF9208
:103100000F931F93CF93DF93CDB7DEB7A1970FB681
:10311000F894DEBF0FBECDBF7C01C42EE52FCB01DE
:10312000D22E19A221E02D1510F02AE0D22E8E0108
:103130000F5D1F4F8D2C912CA12CB12C6C2D7E2F4F
:10314000A50194010E94D81D8C2DD29E80191124B6
:10315000015011098A3014F4805D01C0895CF801C6
:103160008083211531054105510521F0C22EE32F41
:10317000CA01E4CFB801C7010E94F017A1960FB6AB
:10318000F894DEBF0FBECDBFDF91CF911F910F919D
:10319000FF90EF90DF90CF90BF90AF909F908F9077
:1031A0000895CF92DF92EF92FF920F931F93CF93E8
:1031B000DF93EC016A017B012115310579F4E88187
:1031C000F9810190F081E02D642FDF91CF911F9163
:1031D0000F91FF90EF90DF90CF9009942A30310546
:1031E000E9F477FF1AC06DE20E9437188C0144277A
:1031F0005527BA014C195D096E097F092AE0CE01F5
:103200000E947818800F911FDF91CF911F910F912D
:10321000FF90EF90DF90CF9008952AE0B701A601CC
:10322000CE01DF91CF911F910F91FF90EF90DF9032
:10323000CF900C9478189A01AB01662757FD6095E2
:10324000762F0C94D1180F931F93CF93DF93EC013B
:103250009A01AB01662757FD6095762F0E94D11821
:103260008C01CE010E943E18800F911FDF91CF91FB
:103270001F910F9108952115310541F4DC01ED9165
:10328000FC910190F081E02D642F09940C94781842
:103290009A01462F50E060E070E00C943B190F93C8
:1032A0001F93CF93DF93EC010E943B198C01CE0159
:1032B0000E943E18800F911FDF91CF911F910F91B7
:1032C0000895FC01808191810C94981ECF93DF9327
:1032D000EC0188819981009711F00E94981E198253
:1032E00018821D821C821B821A82DF91CF91089561
:1032F0000F931F93CF93DF93EC018B016F5F7F4F91
:10330000888199810E94271F009731F099838883D3
:103310001B830A8381E001C080E0DF91CF911F9180
:103320000F910895CF93DF93EC0188819981892BC8
:1033300029F08A819B818617970760F4CE010E944D
:103340007819882341F08C819D81892B19F4E881BB
:10335000F981108281E0DF91CF910895EF92FF9281
:103360000F931F93CF93DF93EC017B018A01BA0186
:103370000E949219811104C0CE010E94661907C0F3
:103380001D830C83B701888199810E945120CE0151
:10339000DF91CF911F910F91FF90EF900895FC0165
:1033A00011821082138212821582148261157105B6
:1033B00059F0FB0101900020E9F7AF01415051099C
:1033C000461B570B0C94AE1908950F931F93CF9380
:1033D000DF938C01EB01FC0180819181009799F0D2
:1033E000428153812C813D814217530750F06881FF
:1033F00079810E9451208C819D81F801958384837D
:1034000013C00E94981E88819981F801918380835E
:103410008A819B81938382838C819D819583848320
:10342000198218821B821A821D821C82DF91CF9121
:103430001F910F910895CF93DF93EC0186179707A3
:1034400011F00E94E519CE01DF91CF910895CF933D
:10345000DF93EC016115710561F0FB010190002023
:10346000E9F7AF0141505109461B570B0E94AE19B5
:1034700002C00E946619CE01DF91CF9108950F938B
:103480001F93CF93DF93CDB7DEB729970FB6F8948C
:10349000DEBF0FBECDBF8C01862FF80111821082D6
:1034A000138212821582148250E0BE016F5F7F4F3B
:1034B00090E00E94B420BE016F5F7F4FC8010E9460
:1034C000271A29960FB6F894DEBF0FBECDBFDF9145
:1034D000CF911F910F9108950F931F93CF93DF9377
:1034E000CDB7DEB762970FB6F894DEBF0FBECDBF83
:1034F0008C01CB01F8011182108213821282158295
:10350000148250E0BE016F5F7F4F0E948120BE0198
:103510006F5F7F4FC8010E94271A62960FB6F8941A
:10352000DEBF0FBECDBFDF91CF911F910F910895E8
:10353000EF92FF920F931F93CF93DF93EC017B01E8
:103540000C811D816115710511F480E016C04115D3
:10355000510591F0040F151FB8010E94921988239C
:10356000A1F3288139818C819D81B701820F931F3E
:103570000E9451201D830C8381E0DF91CF911F9128
:103580000F91FF90EF900895FB0144815581608178
:1035900071810C94981A6115710559F0FB01019025
:1035A0000020E9F7AF0141505109461B570B0C941D
:1035B000981A80E00895CF93DF9300D0CDB7DEB79F
:1035C00069831A8241E050E0BE016F5F7F4F0E9425
:1035D000981A0F900F90DF91CF910895EF92FF927C
:1035E0000F931F93CF93DF9300D000D0CDB7DEB7FA
:1035F0007C01862F4AE08E010F5F1F4FB80190E0DB
:103600000E948C20F80101900020E9F7AF014150A1
:103610005109401B510BB801C7010E94981A0F9025
:103620000F900F900F90DF91CF911F910F91FF900E
:10363000EF900895EF92FF920F931F93CF93DF9334
:10364000CDB7DEB728970FB6F894DEBF0FBECDBF5B
:103650007C01CB014AE08E010F5F1F4FB8010E9431
:103660008C20F80101900020E9F7AF014150510989
:10367000401B510BB801C7010E94981A28960FB63B
:10368000F894DEBF0FBECDBFDF91CF911F910F9198
:10369000FF90EF900895FC01248135816217730734
:1036A00048F480819181009729F0FC01E60FF71F13
:1036B0008081089580E008950C944B1B0F931F9315
:1036C000CF93DF93EB0141155105E9F02097D9F035
:1036D000FC016481758126173707A0F4621B730B08
:1036E0008A01015011096017710708F48B01FC0170
:1036F00060817181620F731FA801CE010E94582062
:10370000C00FD11F1882DF91CF911F910F910895A3
:10371000CF93DF93FC01848195814817590778F492
:10372000C081D181FB0160817181CE01840F951F21
:103730000E946720009719F08C1B9D0B02C08FEF31
:103740009FEFDF91CF910895BF92CF92DF92EF92DA
:10375000FF920F931F93CF93DF936C017B01EA01DC
:1037600089012417350720F48D2FE901042F182F24
:1037700067E072E0C6010E94CF19D70114968D91BF
:103780009C911597C817D907C8F48017910708F4BA
:103790008C01D701ED91FC911197E00FF11FB080E2
:1037A00010826D917C916C0F7D1FC6010E94271ABB
:1037B000D701ED91FC91E00FF11FB082C601DF91BE
:1037C000CF911F910F91FF90EF90DF90CF90BF901E
:1037D0000895FC0180819181009711F00C940F20D5
:1037E00060E070E0CB01089508955058BB27AA27E8
:1037F0000ED009C1FAD030F0FFD020F031F49F3F55
:1038000011F41EF4EFC00EF4E095E7FBE5C0E92FDC
:103810000BD180F3BA17620773078407950718F076
:1038200071F49EF523C10EF4E0950B2EBA2FA02D56
:103830000B01B90190010C01CA01A0011124FF275D
:10384000591B99F0593F50F4503E68F11A16F04058
:10385000A22F232F342F4427585FF3CF4695379557
:103860002795A795F0405395C9F77EF41F16BA0B1C
:10387000620B730B840BBAF09150A1F0FF0FBB1FCA
:10388000661F771F881FC2F70EC0BA0F621F731F13
:10389000841F48F4879577956795B795F7959E3F70
:1038A00008F0B3CF9395880F08F09927EE0F9795FE
:1038B0008795089504D06894B111D9C00895BCD0FB
:1038C00088F09F5790F0B92F9927B751A0F0D1F009
:1038D000660F771F881F991F1AF0BA95C9F712C093
:1038E000B13081F0C3D0B1E00895C0C0672F782F08
:1038F0008827B85F39F0B93FCCF3869577956795FF
:10390000B395D9F73EF490958095709561957F4F6A
:103910008F4F9F4F0895E89409C097FB3EF4909510
:103920008095709561957F4F8F4F9F4F9923A9F098
:10393000F92F96E9BB279395F69587957795679527
:10394000B795F111F8CFFAF4BB0F11F460FF1BC06B
:103950006F5F7F4F8F4F9F4F16C0882311F096E9FE
:1039600011C0772321F09EE8872F762F05C06623AC
:1039700071F096E8862F70E060E02AF09A95660F65
:10398000771F881FDAF7880F9695879597F908951E
:10399000990F0008550FAA0BE0E8FEEF1616170660
:1039A000E807F907C0F012161306E407F50798F0C8
:1039B000621B730B840B950B39F40A2661F0232BE1
:1039C000242B252B21F408950A2609F4A140A6955D
:1039D0008FEF811D811D089597F99F6780E870E042
:1039E00060E008959FEF80EC089500240A94161675
:1039F000170618060906089500240A9412161306DD
:103A0000140605060895092E0394000C11F488236A
:103A100052F0BB0F40F4BF2B11F460FF04C06F5F86
:103A20007F4F8F4F9F4F089557FD9058440F551F5C
:103A300059F05F3F71F04795880F97FB991F61F030
:103A40009F3F79F087950895121613061406551FA7
:103A5000F2CF4695F1DF08C0161617061806991F13
:103A6000F1CF86957105610508940895E894BB2708
:103A700066277727CB0197F908958ADF08F48FEF3F
:103A800008950BD0C0CFB1DF28F0B6DF18F0952332
:103A900009F0A2CFA7CF1124EACFC6DFA0F3959FEC
:103AA000D1F3950F50E0551F629FF001729FBB2725
:103AB000F00DB11D639FAA27F00DB11DAA1F649FD1
:103AC0006627B00DA11D661F829F2227B00DA11D84
:103AD000621F739FB00DA11D621F839FA00D611D0A
:103AE000221F749F3327A00D611D231F849F600D2B
:103AF000211D822F762F6A2F11249F5750408AF064
:103B0000E1F088234AF0EE0FFF1FBB1F661F771FEF
:103B1000881F91505040A9F79E3F510570F05CCF2F
:103B2000A6CF5F3FECF3983EDCF3869577956795DB
:103B3000B795F795E7959F5FC1F7FE2B880F911D0D
:103B40009695879597F90895991B79E004C0991F78
:103B5000961708F0961B881F7A95C9F780950895E7
:103B6000AA1BBB1B51E107C0AA1FBB1FA617B707A3
:103B700010F0A61BB70B881F991F5A95A9F78095BF
:103B80009095BC01CD01089597FB072E16F4009483
:103B900007D077FD09D00E94B01D07FC05D03EF488
:103BA000909581959F4F0895709561957F4F0895E9
:103BB000A1E21A2EAA1BBB1BFD010DC0AA1FBB1F31
:103BC000EE1FFF1FA217B307E407F50720F0A21BA3
:103BD000B30BE40BF50B661F771F881F991F1A9410
:103BE00069F760957095809590959B01AC01BD013A
:103BF000CF010895EE0FFF1F0590F491E02D099479
:103C0000CF93DF938230910510F482E090E0E09151
:103C1000E104F091E20420E030E0A0E0B0E0309771
:103C200039F14081518148175907B8F048175907B1
:103C300071F482819381109729F013969C938E934F
:103C400012972CC09093E2048093E10427C02115C1
:103C5000310531F04217530718F0A901DB0101C00B
:103C6000EF019A01BD01DF010280F381E02DD7CF82
:103C700021153105F9F0281B390B2430310580F46A
:103C80008A819B816115710521F0FB0193838283F9
:103C900004C09093E2048093E104FE01329644C094
:103CA000FE01E20FF31F8193919322503109398372
:103CB00028833AC02091DF043091E004232B41F4A3
:103CC00020910201309103013093E0042093DF043E
:103CD00020910001309101012115310541F42DB7EA
:103CE0003EB74091040150910501241B350BE09132
:103CF000DF04F091E004E217F307A0F42E1B3F0B62
:103D00002817390778F0AC014E5F5F4F241735074D
:103D100048F04E0F5F1F5093E0044093DF048193FF
:103D2000919302C0E0E0F0E0CF01DF91CF910895E0
:103D3000CF93DF93009709F487C0FC013297138279
:103D40001282C091E104D091E204209781F4208195
:103D50003181280F391F8091DF049091E004821790
:103D6000930779F5F093E004E093DF046DC0DE0182
:103D700020E030E0AE17BF0750F412964D915C91F1
:103D800013979D014115510509F1DA01F3CFB38372
:103D9000A28340815181840F951F8A179B0771F47C
:103DA0008D919C911197840F951F0296918380832A
:103DB00012968D919C9113979383828321153105DF
:103DC00029F4F093E204E093E1043EC0D901139694
:103DD000FC93EE9312974D915D91A40FB51FEA17D6
:103DE000FB0779F480819181840F951F0296D90198
:103DF00011969C938E938281938113969C938E93BC
:103E00001297E0E0F0E08A819B81009719F0FE01B3
:103E1000EC01F9CFCE01029628813981820F931FE0
:103E20002091DF043091E0042817390769F43097B6
:103E300029F41092E2041092E10402C0138212826B
:103E4000D093E004C093DF04DF91CF910895A0E008
:103E5000B0E0EDE2FFE10C949D23EC01CB01209753
:103E600019F40E94001EB8C0FE01E60FF71F9E0164
:103E700022503109E217F30708F4ACC0D9010D91C3
:103E80001C91119706171707B8F00530110508F4B3
:103E90009FC0A801445051094617570708F498C01D
:103EA00002501109061B170B019311936D937C931C
:103EB000CF010E94981E8CC05B01A01AB10A4E016E
:103EC000800E911EA091E104B091E204612C712C4E
:103ED00060E070E0109709F449C0A815B905C9F56C
:103EE000ED90FC901197670142E0C40ED11CCA14FA
:103EF000DB0478F147018A189B08640142E0C40E94
:103F0000D11C1296BC9012971396AC91B5E0CB16CB
:103F1000D10440F0B282A38391828082D9018D9333
:103F20009C9309C00E5F1F4F0E0D1F1DF9011183D9
:103F30000083EB2DFA2F6115710531F0DB0113962B
:103F4000FC93EE93129744C0F093E204E093E104F3
:103F50003FC06D917C9111976616770608F43B017E
:103F6000BD0112960D90BC91A02DB4CF6091DF04DD
:103F70007091E00468157905E9F468167906D0F4C3
:103F800040910001509101014115510541F44DB797
:103F90005EB76091040170910501461B570BE41751
:103FA000F507C0F4F093E004E093DF04F901918396
:103FB00080830EC00E94001E7C01009759F0A8016A
:103FC000BE010E943620CE010E94981EC70104C087
:103FD000CE0102C080E090E0CDB7DEB7EEE00C94F9
:103FE000B923FC0188279927E89421912032E9F32D
:103FF000293010F02E30C8F32B3241F02D3239F435
:10400000689404C00E94AC20820F911D219120531E
:104010002A30C0F31EF4909581959F4F08951F9309
:10402000FC0199278827BC01E89411911032E9F32B
:10403000193010F01E30C8F31B3251F01D3249F414
:10404000689406C00E949720610F711D811D911D0B
:10405000119110531A30B0F33EF4909580957095FD
:1040600061957F4F8F4F9F4F1F910895FB01DC019A
:1040700002C001900D9241505040D8F70895681742
:10408000790768F4FB01DC01E40FF51FA40FB51FED
:1040900002C002900E9241505040D8F708950C94FF
:1040A0003620FB01DC0101900D920020E1F708951C
:1040B000FB01DC014150504048F001900D9200207E
:1040C000C9F701C01D9241505040E0F70895FB012F
:1040D00051915523A9F0BF01DC014D9145174111C4
:1040E000E1F759F4CD010190002049F04D914015C0
:1040F0004111C9F3FB014111EFCF81E090E001973D
:1041000008954532510520F4423010F00C948C2073
:10411000FB011082CB010895BB274A3031F499236B
:1041200022F4BDE2909581959F4F0C94C020592FA9
:10413000482F372F262F660F771F881F991F660F6E
:10414000771F881F991F620F731F841F951F660FAB
:10415000771F881F991F08957AE0979F902D879F5A
:10416000802D910D112408954532510520F44230DF
:1041700010F00C94BF20FB011082CB010895BB27E7
:10418000FB015527AA27880F991FAA1FA41710F013
:10419000A41B83955051B9F7A05DAA3308F0A95D1F
:1041A000A193009779F7B111B1931192CB010C94BF
:1041B000F922AEE0B0E0EFEDF0E20C94A7230D8918
:1041C0001E8986E08C831A8309838FEF9FE79E8385
:1041D0008D83AE01475E5F4F6F89788DCE0101966A
:1041E0000E94FB20EF81F885E00FF11F10822E96D0
:1041F000E4E00C94C323ACE0B0E0E1E0F1E20C9425
:1042000099237C016B018A01FC011782168283814C
:1042100081FFBDC1CE0101964C01F7019381F601EA
:1042200093FD859193FF81916F01882309F4ABC1C0
:10423000853239F493FD859193FF81916F01853229
:1042400029F4B70190E00E940923E7CF512C312CCB
:1042500020E02032A0F48B3269F030F4803259F043
:10426000833269F420612CC08D3239F0803339F407
:10427000216026C02260246023C0286021C027FD61
:1042800027C030ED380F3A3078F426FF06C0FAE048
:104290005F9E300D1124532E13C08AE0389E300DDE
:1042A0001124332E20620CC08E3221F426FD6BC106
:1042B000206406C08C3611F4206802C0883641F4B0
:1042C000F60193FD859193FF81916F018111C1CF1B
:1042D000982F9F7D9554933028F40C5F1F4FFFE378
:1042E000F9830DC0833631F0833771F0833509F0DF
:1042F0005BC022C0F801808189830E5F1F4F442478
:104300004394512C540115C03801F2E06F0E711C1A
:10431000F801A080B18026FF03C0652D70E002C0C7
:104320006FEF7FEFC5012C870E94EE222C018301E5
:104330002C852F77222E17C03801F2E06F0E711CEA
:10434000F801A080B18026FF03C0652D70E002C097
:104350006FEF7FEFC5012C870E94E3222C012C8593
:104360002068222E830123FC1BC0832D90E0481679
:104370005906B0F4B70180E290E00E9409233A9414
:10438000F4CFF50127FC859127FE81915F01B701EC
:1043900090E00E94092331103A94F1E04F1A51083D
:1043A0004114510471F7E5C0843611F0893639F5AE
:1043B000F80127FF07C060817181828193810C5FC2
:1043C0001F4F08C060817181882777FD8095982FE5
:1043D0000E5F1F4F2F76B22E97FF09C090958095E4
:1043E000709561957F4F8F4F9F4F2068B22E2AE0C6
:1043F00030E0A4010E943B23A82EA81844C08537B2
:1044000029F42F7EB22E2AE030E025C0F22FF97F6A
:10441000BF2E8F36C1F018F4883579F0B4C08037DC
:1044200019F0883721F0AFC02F2F2061B22EB4FED3
:104430000DC08B2D8460B82E09C024FF0AC09F2FA9
:104440009660B92E06C028E030E005C020E130E0DB
:1044500002C020E132E0F801B7FE07C0608171813F
:10446000828193810C5F1F4F06C06081718180E063
:1044700090E00E5F1F4FA4010E943B23A82EA818B6
:10448000FB2DFF77BF2EB6FE0BC02B2D2E7FA51464
:1044900050F4B4FE0AC0B2FC08C02B2D2E7E05C01D
:1044A0007A2C2B2D03C07A2C01C0752C24FF0DC053
:1044B000FE01EA0DF11D8081803311F4297E09C0CF
:1044C00022FF06C07394739404C0822F867809F08B
:1044D000739423FD13C020FF06C05A2C731418F4E4
:1044E000530C5718732C731468F4B70180E290E0F2
:1044F0002C870E94092373942C85F5CF731410F434
:10450000371801C0312C24FF12C0B70180E390E0BE
:104510002C870E9409232C8522FF17C021FF03C08E
:1045200088E590E002C088E790E0B7010CC0822FD8
:10453000867859F021FD02C080E201C08BE227FDA0
:104540008DE2B70190E00E940923A51438F4B70169
:1045500080E390E00E9409235A94F7CFAA94F401D3
:10456000EA0DF11D8081B70190E00E940923A1109E
:10457000F5CF332009F451CEB70180E290E00E94DC
:1045800009233A94F6CFF7018681978102C08FEF15
:104590009FEF2C96E2E10C94B523F999FECF92BDE2
:1045A00081BDF89A992780B50895262FF999FECFF5
:1045B0001FBA92BD81BD20BD0FB6F894FA9AF99A40
:1045C0000FBE01960895FC010590615070400110E6
:1045D000D8F7809590958E0F9F1F0895FC0161502C
:1045E000704001900110D8F7809590958E0F9F1F15
:1045F0000895DC01FC01672F71917723E1F7329771
:1046000004C07C916D9370836291AE17BF07C8F3AD
:1046100008950F931F93CF93DF93182F092FEB016A
:104620008B8181FD03C08FEF9FEF20C082FF10C000
:104630004E815F812C813D81421753077CF4E881D4
:10464000F9819F012F5F3F4F39832883108306C074
:10465000E885F985812F0995892B29F72E813F81DE
:104660002F5F3F4F3F832E83812F902FDF91CF917C
:104670001F910F910895FA01AA27283051F1203196
:1046800081F1E8946F936E7F6E5F7F4F8F4F9F4FE6
:10469000AF4FB1E03ED0B4E03CD0670F781F891F28
:1046A0009A1FA11D680F791F8A1F911DA11D6A0FF6
:1046B000711D811D911DA11D20D009F468943F91A9
:1046C0002AE0269F11243019305D3193DEF6CF01A8
:1046D0000895462F4770405D4193B3E00FD0C9F76E
:1046E000F6CF462F4F70405D4A3318F0495D31FDDB
:1046F0004052419302D0A9F7EACFB4E0A69597952E
:10470000879577956795BA95C9F700976105710503
:1047100008959B01AC010A2E06945795479537954D
:104720002795BA95C9F7620F731F841F951FA01DA7
:1047300008952F923F924F925F926F927F928F9245
:104740009F92AF92BF92CF92DF92EF92FF920F9320
:104750001F93CF93DF93CDB7DEB7CA1BDB0B0FB62A
:10476000F894DEBF0FBECDBF09942A8839884888E7
:104770005F846E847D848C849B84AA84B984C8847D
:10478000DF80EE80FD800C811B81AA81B981CE0F74
:10479000D11D0FB6F894DEBF0FBECDBFED01089559
:1047A00010E0CCEED0E004C0FE010E94FC1D229679
:0A47B000CE3ED107C9F7F894FFCF01
:1047BA000000E30480002C0106CB13CB133B004915
:1047CA0054506172616D733A20004F4B005620338A
:1047DA002E322E302D686631205349474E414C64A3
:1047EA0075696E6F202D20636F6D70696C6564202A
:1047FA006174204D617220203420323031362032EB
:10480A00323A34303A35310053796E633A20002017
:10481A002D3E2053796E63466163743A20002C2042
:10482A00436C6F636B3A20002C20546F6C3A200063
:10483A002C20506174744C656E3A20002C205075FF
:10484A006C73653A20002C20002C206D5374617221
:10485A00743A20005369676E616C3A20002E20007A
:10486A00205B005D005061747465726E3A2000200E
:10487A0050002A5B002C0025303258004C4C3D0079
:10488A004C483D00534C3D0053483D00433D004DCC
:10489A005300443D0043503D0053503D004F004DEE
:1048AA0055004D4300000000004916C817CB15E417
:1048BA0015D61527160D0A006E616E00696E660020
:0648CA006F7666002E006F
:00000001FF
